:020000040800F2
:10000000A0070020A501000861100008A30E000849
:100010005D100008690A0008AB1F0008000000001E
:10002000000000000000000000000000B5150008FE
:10003000410C00080000000045140008A11600084B
:10004000BF010008BF010008BF010008BF01000890
:10005000BF010008BF010008BF010008BF01000880
:10006000BF010008BF010008BF010008BF01000870
:10007000BF010008BF010008BF010008BF01000860
:10008000BF010008BF010008BF010008BF01000850
:10009000BF010008BF010008BF010008BF01000840
:1000A000BF010008BF010008BF010008BF01000830
:1000B000BF010008BD17000809190008BF010008AA
:1000C000BF010008BF010008BF010008BF01000810
:1000D000BF010008091D0008BF010008BF0100089A
:1000E000BF010008BF010008BF01000800F002F8CE
:1000F00000F048F80AA090E8000C82448344AAF17A
:100100000107DA4501D100F03DF8AFF2090EBAE877
:100110000F0013F0010F18BFFB1A43F0010318473B
:10012000D4530000F4530000103A24BF78C878C1BB
:10013000FAD8520724BF30C830C144BF04680C60ED
:10014000704700000023002400250026103A28BF35
:1001500078C1FBD8520728BF30C148BF0B60704739
:10016000642900F07D80002070471FB500F0E8FA98
:1001700004000020002103F0B3FD401C60601FBD9F
:1001800010B510BD00F0B7FA1146FFF7EEFF03F00F
:100190000DFC00F0E7FA03B4FFF7F2FF03BC02F036
:1001A00020F900000948804709480047FEE7FEE7BC
:1001B000FEE7FEE7FEE7FEE7FEE7FEE7FEE7FEE717
:1001C00004480549054A064B70470000A51600087B
:1001D000ED000008A0010020A0070020A0030020DF
:1001E000A0030020704700000FB41CB5074B06AAFF
:1001F0007B4469460090059800F0D1F900206946DB
:1002000000F0E0F91CBC5DF814FB0000D103000015
:1002100070B5044685690068C10601D5302600E046
:100220002026C00707D070BDD4E901213046904791
:10023000206A401C20626D1EF6D570BD70B5044664
:1002400085690078C00707D170BDD4E9012120205D
:100250009047206A401C20626D1EF6D570BD0000DC
:100260002DE9F0410646002410687529314616A58F
:1002700010D0AFF30080002802DA404213A507E057
:1002800031688A0701D512A502E0490704D511A5F6
:10029000012401E0AFF3008000210A2206F12407C7
:1002A00009E0B0FBF2FCB0FBF2F302FB1C003030C3
:1002B00078541846491C0028F3D123462A46304674
:1002C000BDE8F04100F00CB9000000002D00000076
:1002D0002B000000200000002DE9F0474FF0000A3D
:1002E00089460446C0F820A02046E16888470028D7
:1002F00076D0252806D0D4E901219047206A401CF9
:100300002062F1E7E168204600258847C4F81CA078
:1003100006460027C4F818A02A2E09D0304602F05D
:1003200059F838B304EB8708303EC8F8186019E074
:1003300059F8041B204604EB87029161E168884765
:10034000012F064618D1E069002820DA25F02005A3
:100350001DE0D8F8180000EB800006EB40003038B4
:10036000C8F818002046E1688847064602F032F8CF
:100370000028EED1012F0AD02E2E08D12046E168A8
:1003800088477F1C0646022F45F02005C4DBA06984
:10039000002803DA404245F00105A061E80701D0DA
:1003A00025F01005B6B1A6F14100192802D8203673
:1003B00045F400654A463146204625604D46FFF724
:1003C000CFFE58B1012806D0ED1D25F0070000F141
:1003D000080989E704E005F1040985E730468AE762
:1003E000206ABDE8F08770B5064600F075F804682D
:1003F000054630460A22002100F0E9F82C6070BD65
:1004000030B505460B462A4613F8014B12F8010B8E
:1004100008B1A042F8D01CB1002802D06D1CF1E751
:10042000284630BD421E12F8013F002BFBD111F8C7
:10043000013B002B02F8013BF9D170474FF000025D
:100440000429C0F0128010F0030C00F01B80CCF1E6
:10045000040CBCF1020F18BF00F8012BA8BF20F854
:10046000022BA1EB0C0100F00DB85FEAC17C24BFA8
:1004700000F8012B00F8012B48BF00F8012B704752
:100480004FF0000200B5134694469646203922BF2D
:10049000A0E80C50A0E80C50B1F12001BFF4F7AF78
:1004A000090728BFA0E80C5048BF0CC05DF804EB5A
:1004B000890028BF40F8042B08BF704748BF20F8C8
:1004C000022B11F0804F18BF00F8012B70477047C6
:1004D0007047704770470000004870473C0100209B
:1004E0002DE9F0470D4699469246044600F124084E
:1004F0000168880604D5E06921F01001216000E060
:100500000120A84201DD471B00E00027A1697A19FC
:1005100002EB0900081AA0612078C00602D4204628
:10052000FFF776FE002608E0D4E901211AF806005C
:100530009047206A401C761C20624E45F4DB2078F0
:10054000C0060AD52046FFF763FE06E0D4E9012184
:1005500030209047206A401C2062381EA7F1010716
:10056000F4DC07E0D4E9012118F805009047206A7F
:10057000401C2062281EA5F10105F3DC2046FFF790
:100580005DFE2078000602D50220BDE8F08701203C
:10059000FBE7000001694A1C02610878704700B55A
:1005A0008FB0CDE901310021059105497944CDE9AC
:1005B000031011466846FFF78FFE0FB000BD000024
:1005C000E5FFFFFF0A6802F8010B0A6070472DE99A
:1005D000F04791460F4680460446002614F8015B1A
:1005E0002DB100F031F80068405DC007F6D12B2D29
:1005F00002D02D2D18D0641E4A463946204600F000
:100600002BF827B13968A14201D1C7F800804FF01B
:10061000020471050BD54042002803DDFFF75CFFA3
:100620000460A007BDE8F08746F48066E4E7002890
:10063000F8DAFFF751FF04606FF00040F2E70000C6
:10064000004870473C01002010B500F079F8001D0B
:1006500010BD00BF8D3600002DE9F05F82461546C3
:100660008B4600270AF10104B9460078302801D0F2
:100670009DB113E014F8010B0127782803D0582806
:1006800001D045B10AE00DB1102D07D1002714F8B3
:10069000010B102502E0082500E00A250026B046DF
:1006A0000EE005FB080005FB06F101271FFA80F8A4
:1006B00001EB1046B6F5803F00D3B94614F8010BA4
:1006C000294600F041F80028EBDABBF1000F05D015
:1006D0000FB1641E00E05446CBF80040B9F1000FA2
:1006E00006D0FFF7F9FE02210160C81EBDE8F09FA9
:1006F00048EA0640FAE77546FFF7A2FFAE46050056
:100700006946534620F00700854618B020B5FFF72C
:1007100057FDBDE820404FF000064FF000074FF0B6
:1007200000084FF0000B21F00701AC46ACE8C0090F
:10073000ACE8C009ACE8C009ACE8C0098D46704718
:10074000004870475C0100203A2800D2303820F081
:100750002002412A01D3A2F13700884201D34FF091
:10076000FF3070470446AFF300802046FFF713FDCB
:100770004FF0013C50F8042B51F8043B9A4221D130
:10078000A2EB0C03934313EACC1317D150F8042BBC
:1007900051F8043B9A4215D1A2EB0C03934313EAA0
:1007A000CC130BD150F8042B51F8043B9A4209D1D9
:1007B000A2EB0C03934313EACC13DBD04FF0000001
:1007C000704700BFD01A01BAB1FA81F101F01801E7
:1007D00022FA01F0CB40C1F12001DBB2C0B2C01A55
:1007E0002CFA01F3D11A914311EAC311E6D17047F3
:1007F00021B1826842F00102826003E0826822F047
:10080000010282607047000010B50446124884421D
:1008100008D10121401500F053FE0021601500F0C1
:100820004FFE17E00D48844208D10121001500F069
:1008300047FE0021201500F043FE0BE008488442EB
:1008400008D10121C80300F03BFE00214FF4004015
:1008500000F036FE10BD00000024014000280140D9
:10086000003C0140014600208A6802F004020AB1FF
:10087000012000E0002070470146C86C80B270473C
:100880000246002013680B400BB1012000E000205D
:100890007047014600208A6802F008020AB1012070
:1008A00000E000207047000030B502460020002321
:1008B00050680F4C20400D790C6844EA0524204311
:1008C000506090680B4C2040D1E902542C434D7984
:1008D00044EA450420439060D06A20F470000C7C08
:1008E000641EE4B2234340EA0350D06230BD0000EE
:1008F000FFFEF0FFFDF7F1FFF0B504460D460020C6
:100900000021092D11DDE068A5F10A0606EB460776
:10091000072606FA07F18843A5F10A0606EB460604
:1009200003FA06F10843E0600CE0206905EB450797
:10093000072606FA07F1884305EB450603FA06F198
:1009400008432061072A0FDA606B561E06EB860704
:100950001F2606FA07F18843561E06EB860605FA9F
:1009600006F10843606322E00D2A0FDA206BD61FE0
:1009700006EB86071F2606FA07F18843D61F06EB0B
:10098000860605FA06F10843206310E0E06AA2F14A
:100990000D0606EB86071F2606FA07F18843A2F12B
:1009A0000D0606EB860605FA06F10843E062F0BD87
:1009B000816841F008018160704721B1826842F48A
:1009C000A002826003E0826822F4A0028260704785
:1009D000816841F0040181607047000000B587B074
:1009E00001214FF4017000F05BFD4FF4004000F076
:1009F0002BFD7020ADF8040000208DF8070001A940
:100A0000174800F01EF91748FFF7FEFE002002907D
:100A10008DF80C008DF80D004FF46020049000203C
:100A2000059001208DF8180002A90E48FFF73CFF41
:100A300001210C48FFF7DCFE0A48FFF7B9FF00BFB1
:100A40000848FFF726FF0028FAD10648FFF7C0FF45
:100A500000BF0448FFF706FF0028FAD107B000BD29
:100A6000000801400024014000BFFEE710B500214E
:100A7000014800F06FFF10BD0008004010B50024D1
:100A8000002000F045F804E0601CC4B2012001F031
:100A900037FD20210E4800F0A7F908B1642CF3DBE4
:100AA000642C01DB012010BD002404E0601CC4B2F2
:100AB000012001F025FD2021054800F095F908B935
:100AC000642CF3DB642C01DB0120ECE70020EAE777
:100AD000000C014008B50121082000F0E1FC2020B5
:100AE000ADF8000010208DF8030003208DF80200FF
:100AF0006946064800F0A5F82021044800F07FF977
:100B000000F088F8FFF7BAFF08BD0000000C0140B4
:100B100038B504464CB12020ADF8000003208DF814
:100B2000020010208DF8030005E02020ADF8000041
:100B300004208DF803006946014800F082F838BDB2
:100B4000000C014010B5002404E0601CC4B2012078
:100B500001F0D6FC2021104800F046F908B1642CC1
:100B6000F3DB002404E0601CC4B2012001F0C8FCE7
:100B70002021094800F038F908B9642CF3DB28205B
:100B800001F0BEFC2021044800F02EF908B101203C
:100B900010BD0020FCE70000000C014070B50024EF
:100BA000002506E06006040EFFF7CCFF0443681C36
:100BB000C5B2082DF6DB204670BD7CB505460E4655
:100BC00000F028F8FFF75AFFF8B9002405E0FFF716
:100BD000E5FF0DF80400601CC4B2052CF7DB9DF89E
:100BE00000009DF8011008449DF8021008449DF88B
:100BF000031008449DF80410884208D19DF80000B5
:100C000030709DF80200287001E001207CBD0020BA
:100C1000FCE7000010B50120FFF77AFF202107480C
:100C200000F0EBF8142001F023FC2021034800F031
:100C3000E6F80D2001F064FC10BD0000000C01403E
:100C400070472DE9F04102460025002600200023D0
:100C50000024002791F803C00CF00F0591F803C0A1
:100C60000CF0100CBCF1000F03D091F802C04CEA5C
:100C7000050591F800C0BCF1000F31D014680020C8
:100C80002BE04FF0010C0CFA00F3B1F800C00CEAB5
:100C900003069E4220D183004FF00F0C0CFA03F79D
:100CA000BC4305FA03FC4CEA040491F803C0BCF110
:100CB000280F06D14FF0010C0CFA00FCC2F814C04A
:100CC0000AE091F803C0BCF1480F05D14FF0010CC8
:100CD0000CFA00FCC2F810C0401C0828D1D31460E4
:100CE000B1F800C0BCF1FF0F34DD546800202EE0E5
:100CF00000F1080C4FF0010808FA0CF3B1F800C03D
:100D00000CEA03069E4221D183004FF00F0C0CFA2F
:100D100003F7BC4305FA03FC4CEA040491F803C052
:100D2000BCF1280F05D100F1080C08FA0CF8C2F844
:100D3000148091F803C0BCF1480F07D100F1080CF2
:100D40004FF0010808FA0CF8C2F81080401C08287F
:100D5000CED35460BDE8F081F0B50A4600230024EC
:100D60000021002500F00046B6F1004F02D11D4ED3
:100D7000F16901E01B4E7168C0F3034583B200F4D2
:100D80004016B6F5401F08D121F07061154E766807
:100D900026F07066134F7E6012E000F48016B6F500
:100DA000801F06D1032606FA05F4A14341F07061C5
:100DB00006E0460D360103FA06F6B14341F07061D4
:100DC00022B1460D360103FA06F6314300F0004623
:100DD000B6F1004F02D1034EF16101E0014E7160A6
:100DE000F0BD0000000001400246002093680B4067
:100DF0000BB1012000E000207047416170470161A4
:100E000070470AB1016100E04161704710B500BF51
:100E1000094800884FF47A7100FB01F4074800F09C
:100E2000A9FE04440020054924310880322001F045
:100E30001FFB204610BD00001400002000080040E9
:100E400010B504460723012221460948FFF754FD47
:100E500001210748FFF7B1FD00BF02210448FFF759
:100E60000FFD0028F9D00248FFF706FD10BD000075
:100E7000002401402DE9F04107460C4600250026DC
:100E800008E03846FFF7DCFF0544052001F0F0FAE2
:100E9000701CC6B2A642F4DBB5FBF4F080B2BDE82C
:100EA000F08100BFFEE700002DE9F84F4FF0000A87
:100EB0000024A346A14631E0012021490860142006
:100EC00001F01EFB00201F49C1F8AC0100BF1C4807
:100ED000843800680028FAD000F0A2FA641C00BF31
:100EE0001748843800680128FAD0FFF7BFFDFFF7E4
:100EF0008DFF8246504603F091F9009003F0E4F82C
:100F000007460022104B02F033FF054602F0FEFEBA
:100F100083464946584603F003F98146052CCBD158
:100F2000484603F0D1F807460022084B02F020FFA4
:100F3000054602F0EBFE83465846BDE8F88F0000F8
:100F4000AC8121420080214200004D40000014404D
:100F50001FB50121082000F0A3FA4FF40060ADF89E
:100F6000000003208DF8020010208DF80300694670
:100F70001F48FFF766FE4FF400611D48FFF73DFF75
:100F80004FF48060ADF8000004208DF8030069463E
:100F90001748FFF756FE4FF480611548FFF72DFF05
:100FA0000121042000F05CFA124800F0EFFC40F24E
:100FB000E730ADF808004720ADF804000020ADF898
:100FC0000A00ADF8060001A90A4800F04BFE012115
:100FD000084800F0B9FC01221146064800F0DEFD89
:100FE00002F074FA0021034800F0B4FC1FBD0000B9
:100FF000000C01400008004008B50121182000F055
:101000004FFA0121084600F04BFA01211048FFF782
:10101000A3FE4FF20100ADF8000048208DF8030058
:1010200069460C48FFF70DFE4FF40050ADF8000084
:1010300010208DF8030003208DF802006946064851
:10104000FFF7FFFD4FF400510348FFF7D6FE08BD40
:1010500000023000000C01400010014000BFFEE71C
:10106000704710B54FF4A06000F03AF810BD0000D2
:1010700070B5002100230F22C47804B3154C2468F6
:1010800004F4E064C4F5E064210AC1F10403CA4039
:10109000447804FA03F184781440214309010E4C8A
:1010A0000678A155047804F01F050124AC400578AA
:1010B0006D11AD0005F1E025C5F8004109E00478A7
:1010C00004F01F050124AC40044D0678761145F864
:1010D000264070BD0CED00E000E400E080E100E09F
:1010E00002490143024A1160704700000000FA05FE
:1010F0000CED00E070B500240EE00021204600F069
:10110000DAF8002504E0002000F07AF9681CC5B286
:10111000802DF8DB601CC4B2082CEEDB70BD000033
:1011200008B50121082000F0BBF914208DF8030058
:1011300003208DF80200C020ADF800006946074882
:10114000FFF77FFD012240210448FFF75AFE0122EC
:1011500080210248FFF755FE08BD0000000C014049
:1011600070B50546002413E08020204100EA050206
:1011700080210E48FFF745FE012240210B48FFF772
:1011800040FE002240210948FFF73BFE601CC4B22C
:10119000082CE9DB012240210448FFF732FE00223F
:1011A00040210248FFF72DFE70BD0000000C0140F9
:1011B00010B5012280210948FFF723FE01224021BA
:1011C0000648FFF71EFE002280210448FFF719FEA3
:1011D000002240210148FFF714FE10BD000C014021
:1011E00010B5002280210748FFF70BFE01224021A5
:1011F0000448FFF706FE012280210248FFF701FEA6
:1012000010BD0000000C014070B5002406E0002570
:1012100000E06D1CB5F57A7FFBD3641CB4F57A7FD2
:10122000F5D3FFF77DFFAE2000F0DAF8D52000F00F
:10123000D7F8802000F0D4F8A82000F0D1F83F20A3
:1012400000F0CEF8D32000F0CBF8002000F0C8F872
:10125000402000F0C5F8A12000F0C2F8C82000F03E
:10126000BFF8DA2000F0BCF8122000F0B9F88120B5
:1012700000F0B6F8CF2000F0B3F8D92000F0B0F8B5
:10128000F12000F0ADF8DB2000F0AAF8302000F0EB
:10129000A7F8A42000F0A4F8A62000F0A1F88D2063
:1012A00000F09EF8142000F09BF8AF2000F098F8B2
:1012B000FFF720FF70BD70B505460C4645F0B00045
:1012C00000F08EF8102141EA141000F089F804F0C3
:1012D0000F0000F085F870BD2DE9F04105460E467F
:1012E0001746721ED206110E6A1E5206100EFFF726
:1012F000E2FF002409E0A7F12001134A02EB0111EB
:10130000085D00F07DF8601CC4B2082CF3DB721E8F
:10131000D206110E6A1E012303EB4202D0B2FFF780
:10132000CAFF00240BE0A7F12001074A02EB0112DB
:1013300004F10801505C00F063F8601CC4B2082C92
:10134000F1DBBDE8F0810000C24300082DE9F04167
:1013500006460F4615466806050E7A1E1207110E40
:10136000721E5206100EFFF7A6FF002407E0114977
:1013700001EB4511085D00F043F8601CC4B2102C6D
:10138000F5DB7A1E1207110E721E012303EB4202D7
:10139000D0B2FFF790FF002408E0064A691C02EB78
:1013A0004111085D00F02CF8601CC4B2102CF4DB75
:1013B000BDE8F081B24900082DE9F04107460E462C
:1013C0001546002407E02A5D3019C1B23846FFF700
:1013D00083FF601CC4B2285D0028F4D1BDE8F08111
:1013E00010B50446FFF7E4FE7820FFF7B9FE0020B1
:1013F000FFF7B6FE2046FFF7B3FEFFF7F1FE10BD84
:1014000010B50446FFF7D4FE7820FFF7A9FE402070
:10141000FFF7A6FE2046FFF7A3FEFFF7E1FE10BD93
:1014200010B50021054800F01AFC0020044908808E
:101430000121024800F08EFA10BD000000080040B3
:10144000140000207047000001460020034A506845
:1014500020F44040084350607047000000100240F4
:1014600029B1064AD2690243044BDA6104E0034A17
:10147000D2698243014BDA617047000000100240DC
:1014800029B1064A12690243044B1A6104E0034A77
:1014900012698243014B1A6170470000001002403C
:1014A00029B1064A92690243044B9A6104E0034A57
:1014B00092698243014B9A6170470000001002401C
:1014C00029B1064AD2680243044BDA6004E0034AB9
:1014D000D2688243014BDA6070470000001002407E
:1014E00030B500210022002400232D4D6D6805F049
:1014F0000C0121B1042905D0082923D105E0294D8B
:10150000056022E0274D05601FE0254D6D6805F45C
:101510007012234D6D6805F48034022505EB92426C
:101520001CB9214D554305600BE01D4D6D6805F458
:1015300000351DB11C4D5543056002E0194D554362
:10154000056002E0174D056000BF00BF144D6D68D7
:1015500005F0F0010909154D6B5C0568DD4045603B
:101560000F4D6D6805F4E061090A104D6B5C45682C
:10157000DD4085600A4D6D6805F46051C90A0B4D68
:101580006B5C4568DD40C560054D6D6805F4404104
:10159000890B074D6B5CC568B5FBF3F5056130BD84
:1015A0000010024000127A0000093D0000000020F7
:1015B00010000020704710B500F002F810BD0000C8
:1015C0000CB50020019000903348006840F4803052
:1015D0003149086000BF3048006800F400300090D6
:1015E0000198401C0190009818B90198B0F5A06FBF
:1015F000F1D12948006800F4003010B101200090BA
:1016000001E0002000900098012843D123480068A1
:1016100040F01000214908600846006820F00300EF
:1016200008600846006840F0020008601A484068F8
:10163000194948600846406848600846406840F4D8
:10164000806048600846406820F47C104860084686
:10165000406840F4E81048600846006840F0807038
:10166000086000BF0C48006800F000700028F9D046
:101670000948406820F00300074948600846406870
:1016800040F00200486000BF0348406800F00C00D2
:101690000828F9D10CBD00000010024000200240D3
:1016A0007047000010B51348006840F00100114970
:1016B000086008464068104908400E4948600846DE
:1016C00000680E4908400B4908600846006820F48D
:1016D000802008600846406820F4FE0048604FF40F
:1016E0001F008860FFF767FF4FF000600449086043
:1016F00010BD0000001002400000FFF8FFFFF6FEE2
:1017000008ED00E030B589B004460D460121C8025D
:10171000FFF7C6FE01210420FFF7C2FE4FF48070E0
:10172000ADF8200018208DF8230003208DF822004A
:1017300008A92048FFF785FAADF81840ADF8145015
:101740000020ADF81A00ADF8160005A91A4800F0FF
:1017500089FA7020ADF804000120ADF80600ADF85C
:101760000A400220ADF80C0001A9134800F020FA4D
:101770000121114800F0FAF819208DF8000002202C
:101780008DF8010000208DF8020001208DF8030083
:101790006846FFF76DFC0821074800F055FA012163
:1017A000054800F0C5F80121034800F0D3F809B05E
:1017B00030BD000000080140002C014010B501219F
:1017C0002F4800F0DAF9002859D001212C4800F008
:1017D000BEF82C480088401C2A4908802A48008806
:1017E000401C2949088029480088401C2749088056
:1017F00024480088B0F5967F08DB00202149088046
:101800002348007880F00100214908701F480088B3
:1018100040F6B831884208DB00201C4908801D488A
:10182000007880F001001B49087017480088B0F567
:101830007A7F24DB002014490880012016490870B3
:101840001648006890B916480088401C00B2144938
:101850000880084600883C2811D1002008801148E3
:101860000088401C00B20F49088008E00B4800685F
:10187000012804D100200A4908800A49088010BDC7
:101880000004004056000020580000205A000020AC
:101890004400002043000020450000200081214238
:1018A00024000020260000207FB505460C460121BB
:1018B0000220FFF7D5FDADF80850ADF80440002038
:1018C000ADF80A00ADF8060001A90E4800F0CAF90B
:1018D000012211460B4800F061F91D208DF800002F
:1018E00001208DF8010002208DF8020001208DF802
:1018F00003006846FFF7BCFB0121024800F02AF80C
:101900007FBD00000004004010B50121064800F032
:1019100034F940B10121044800F019F80348008867
:10192000401C0249088010BD00080040140000203F
:1019300021B1028842F08002028004E002884FF662
:101940007F731A4002807047CA4302827047CA43BD
:101950000282704721B1028842F00102028004E055
:1019600002884FF6FE731A400280704731B1B0F81A
:10197000442042F40042A0F8442005E0B0F844209E
:10198000C2F30E02A0F844207047000010B50446D0
:101990006848844208D10121C014FFF791FD00215D
:1019A000E014FFF78DFDC4E0B4F1804F08D10121B0
:1019B0000846FFF765FD00210120FFF761FDB8E053
:1019C0005D48844208D101210220FFF759FD002122
:1019D0000220FFF755FDACE05848844208D10121B0
:1019E0000420FFF74DFD00210420FFF749FDA0E092
:1019F0005348844208D101210820FFF741FD00210E
:101A00000820FFF73DFD94E04E48844208D10121B3
:101A10001020FFF735FD00211020FFF731FD88E091
:101A20004948844208D101212020FFF729FD0021E7
:101A30002020FFF725FD7CE04448844208D10121A5
:101A40004014FFF73DFD00216014FFF739FD70E001
:101A50003F48844209D10121C804FFF731FD00212C
:101A60004FF40020FFF72CFD63E03A48844209D18F
:101A700001210805FFF724FD00214FF48010FFF736
:101A80001FFD56E03448844209D101214805FFF783
:101A900017FD00214FF40010FFF712FD49E02F4819
:101AA000844208D101214020FFF7EAFC00214020B8
:101AB000FFF7E6FC3DE02A48844208D1012180205E
:101AC000FFF7DEFC00218020FFF7DAFC31E025483B
:101AD000844208D101218015FFF7D2FC0021A01516
:101AE000FFF7CEFC25E02048844209D101210804FB
:101AF000FFF7E6FC00214FF48030FFF7E1FC18E02F
:101B00001A48844209D101214804FFF7D9FC002179
:101B10004FF40030FFF7D4FC0BE01548844208D1A5
:101B200001218804FFF7CCFC00214FF48020FFF74F
:101B3000C7FC10BD002C014000040040000800401C
:101B4000000C004000100040001400400034014030
:101B5000004C01400050014000540140001800407A
:101B6000001C0040002000400040014000440140B3
:101B7000004801400146888C704730B5024600207D
:101B800000230024158A05EA0103958905EA01046A
:101B900013B10CB1012000E0002030BD1AB18389DF
:101BA0000B43838102E083898B438381704700006C
:101BB00070B5002400220023058C4FF6FE763540D8
:101BC0000584028C8388048B4FF68F752C40B51EDC
:101BD0002C400D882C43751E2A400D892A434D88C0
:101BE0002A43144DA8420BD0134DA84208D0134DE0
:101BF000A84205D0124DA84202D0124DA84213D1DE
:101C00004FF6F7752A404D892A434FF6FB752A4057
:101C10008D882A434FF6FF652B404FF6FF552B402A
:101C20008D892B43CD892B4383800483CD88858682
:101C3000028470BD002C014000340140004001408E
:101C400000440140004801400A460021018B4FF644
:101C5000F77319401143018370478186704781846F
:101C600070470000002202881D4B98420ED01D4B89
:101C700098420BD0B0F1804F08D01B4B984205D052
:101C80001A4B984202D01A4B984204D14FF68F73E8
:101C90001A404B881A43174B984207D0164B98426C
:101CA00004D04FF6FF431A40CB881A4302808B883A
:101CB00083850B8803850A4B98420BD0094B9842C9
:101CC00008D00E4B984205D00D4B984202D00D4BD8
:101CD000984201D10B7A038601238382704700006A
:101CE000002C014000340140000400400008004086
:101CF000000C004000100040001400400040014073
:101D0000004401400048014010B540F225510E4802
:101D100000F08AF890B10D480068782802D30020BE
:101D20000A490860084800F03BF9C1B20748026858
:101D30000068401C054B18600548815440F225514D
:101D4000014800F007F810BD003801408000002075
:101D5000C400002010B50022002340F66A14A142FE
:101D600000D100BF0A1201249440A3B2DC430480D6
:101D700010BD21B1828942F40052828104E082893F
:101D80004DF6FF731A4082817047000010B504467B
:101D90002048844209D101218803FFF791FB0021EB
:101DA0004FF48040FFF78CFB32E01B48844209D19E
:101DB00001214804FFF764FB00214FF40030FFF7D6
:101DC0005FFB25E01548844209D101218804FFF713
:101DD00057FB00214FF48020FFF752FB18E010481A
:101DE000844209D10121C804FFF74AFB00214FF4C6
:101DF0000020FFF745FB0BE00A48844208D101218F
:101E00000805FFF73DFB00214FF48010FFF738FB7A
:101E100010BD000000380140004400400048004070
:101E2000004C00400050004070B5024600240023E2
:101E30000025002040F66A16B14200D100BFC1F370
:101E4000421501F01F03012606FA03F3012D02D10A
:101E50009689334006E0022D02D1168A334001E014
:101E6000968A33400C12012606FA04F41688344090
:101E700013B10CB1012000E0002070BDF0B50346A5
:101E8000002400260025002040F66A17B94200D140
:101E900000BF1846C1F3421401F01F06012707FADC
:101EA00006F5012C01D10C3004E0022C01D11030D8
:101EB00000E014301AB107682F43076002E007689A
:101EC000AF430760F0BD00002DE9F04786B005463E
:101ED0000E460024A24600BFA1460027B08900B1EB
:101EE00000BF2F462C8A4CF6FF700440F088044354
:101EF0002C82AC894EF6F3100440B0883189084337
:101F0000718908430443AC81AC8A4FF6FF4004401A
:101F1000B0890443AC8201A8FFF7E2FA1F48874268
:101F200002D1DDF810A001E0DDF80CA0A88900F4D2
:101F3000004040B10AEBCA0000EB0A1031684900CA
:101F4000B0FBF1F807E00AEBCA0000EB0A103168B9
:101F50008900B0FBF1F86420B8FBF0F0040120091F
:101F6000642101FB1089A88900F4004040B13220AF
:101F700000EBC900B0FBF1F000F00700044308E0FB
:101F8000322000EB09106421B0FBF1F000F00F00EB
:101F900004432C8106B0BDE8F08700000038014002
:101FA00001468888C0F30800704700BFFEE70000C4
:101FB00070B598B00024002600201790D348006820
:101FC00000287DD00A2000F053FAD1A1D248FEF7B4
:101FD00017FA002832D0CEA1CF48FEF711FA0446F6
:101FE00003E0641C0A2000F043FA20783028F8DB74
:101FF00020783928F5DC00250CE0207817A9485511
:10200000681CC5B2641C20782C2800D108E00A2086
:1020100000F02EFA2078302802DB20783928ECDD19
:1020200000BF2C2017A9485517A8FEF7DCF9064673
:10203000002E03DB632E01DCB8490E70B8A1B64850
:10204000FEF7DEF990B3B6A1B348FEF7D9F904461E
:1020500003E0641C0A2000F00BFA20783028F8DB3B
:1020600020783928F5DC00250CE0207817A94855A0
:10207000681CC5B2641C20782C2800D108E00A2016
:1020800000F0F6F92078302802DB20783928ECDDE2
:1020900000BF2C2017A9485517A8FEF7A4F906463B
:1020A000002E03DB632E01DC9F4806609FA19A4847
:1020B000FEF7A6F990B39DA19748FEF7A1F900E0BD
:1020C000F3E0044603E0641C0A2000F0D1F9207814
:1020D0003028F8DB20783928F5DC00250CE0207862
:1020E00017A94855681CC5B2641C20782C2800D15B
:1020F00008E00A2000F0BCF92078302802DB2078C4
:102100003928ECDD00BF2C2017A9485517A8FEF789
:102110006AF90646002E01DB86490E8086A17E48BC
:10212000FEF76EF990B384A17B48FEF769F9044687
:1021300003E0641C0A2000F09BF920783028F8DBCB
:1021400020783928F5DC00250CE0207817A94855BF
:10215000681CC5B2641C20782C2800D108E00A2035
:1021600000F086F92078302802DB20783928ECDD71
:1021700000BF002017A9485517A8FEF734F90646F6
:10218000002E03DB632E01DC6D490E806DA16248D9
:10219000FEF736F990B36BA15F48FEF731F90446BC
:1021A00003E0641C0A2000F063F920783028F8DB93
:1021B00020783928F5DC00250CE0207817A948554F
:1021C000681CC5B2641C20780D2800D108E00A20E4
:1021D00000F04EF92078302802DB20783928ECDD39
:1021E00000BF002017A9485517A8FEF7FCF80646BF
:1021F000002E03DB632E01DC54490E805448007826
:10220000F0BB54A14448FEF7FBF828B153480078CE
:1022100080F00100514908705048007801283DD1F4
:102220004FA13D48FEF7ECF8C8B101204D490860C8
:10223000502000F01DF900204B49C1F8B4014B4873
:10224000008800F5FA7000B2484908800846B0F9E5
:102250000000B0F5486F02DB40F67F40088044A1E3
:102260002D48FEF7CDF858B101203E4908605020B6
:1022700000F0FEF800203C49C1F8B4013B4800E002
:102280000CE00088A0F5FA7000B2384908800846D2
:10229000B0F90000002801DA0020088078211E48EB
:1022A000FEF7CCF80020194908603348007801286F
:1022B0002AD1002030490870502103A8FEF7E0F829
:1022C0002E48B0F900002E49B1F900102D4AB2F99C
:1022D0000020CDE9002102902B4803782B4802789A
:1022E0002BA103A8FDF780FF1C48007820B935A179
:1022F00003A8FEF797F803E034A103A8FEF792F8CD
:10230000FF2103A801F0C4FC18B070BD80000020BC
:1023100074656D703A000000C40000202C0000209D
:1023200068756D693A0000003000002074696D65C1
:102330003A000000360000206362733A000000009B
:10234000340000207365746C3A00000038000020EF
:10235000540000206D6F6465000000004200002002
:1023600061646400B401224200002242280000207F
:102370006465637200000000450000202600002014
:1023800022000020200000202B0000202A00002036
:102390002474656D703A2564232C2468756D693A40
:1023A0002564232C246C696768743A2564232C2CDB
:1023B000246362733A2564232C2474696D653A257D
:1023C000642300002C6175746F0000002C6D616E39
:1023D00075616C0030380A2801D201207047002056
:1023E000704700BF704710B5024600200BE0135C39
:1023F00003F00F03145C241104EB840403EB440387
:102400001354431CD8B28842F1DB10BD30B50246EC
:1024100000200EE0135C0A2493FBF4F504FB153353
:10242000145C0A2594FBF5F443EA04131354431C8B
:10243000D8B28842EEDB30BD094800680949B0FBDC
:10244000F1F0094908700846007800EB4001C1EB43
:10245000C0104FF6FF7101EAC000044908807047C0
:102460006000002000127A00740000207600002036
:1024700001461F4A12884A434FF0E0235A61002266
:102480009A611A46126942F001021A6100BF4FF0C8
:10249000E0221069174A128B92B1174A1268521C37
:1024A000154B1A601A4612684AF6C8739A4207D941
:1024B0000022114B1A60114A1268521C0F4B1A600D
:1024C00000F001021AB100F48032002ADFD00B4A7A
:1024D0001268B2F5966FDAD84FF0E022126922F056
:1024E00001024FF0E0231A6100229A617047000058
:1024F00076000020A8000020780000207C0000204A
:102500000146114A12784A434FF0E0235A610022F3
:102510009A611A46126942F001021A6100BF4FF037
:10252000E022106900F001021AB100F48032002AA2
:10253000F5D04FF0E022126922F001024FF0E023C3
:102540001A6100229A6170477400002010B56D482E
:102550000078002858D1002203210120FEF7F6FE62
:10256000012205211046FEF7F1FE0222072101207B
:10257000FEF7ECFE64A201210220FEF71DFF0322FC
:1025800011460220FEF7E2FE042205210220FEF79A
:10259000DDFE052207210220FEF7D8FE01F0CCFA6D
:1025A0000F2201210320FEF7D1FE10220221032079
:1025B000FEF7CCFE112203210846FEF7C7FE1222C9
:1025C00004210320FEF7C2FE3A2209210320FEF770
:1025D00083FE132201210420FEF7B8FE14220221FB
:1025E0000420FEF7B3FE152203210420FEF7AEFE01
:1025F000162204210846FEF7A9FE3A2209210420EA
:10260000FEF76AFE00F0B8FD3E480078012877D159
:10261000172201210846FEF799FE18220221012007
:10262000FEF794FE192203210120FEF78FFE1A22E5
:1026300004210120FEF78AFE34A209210120FEF7C1
:10264000BBFE00F06DF81D2201210220FEF77EFE88
:102650002FA203210220FEF7AFFE1E22042102203A
:10266000FEF774FE3A2209210220FEF735FE2AA267
:102670000A210220FEF7A0FE00F0A8FD2922012178
:102680000320FEF763FE22A203210846FEF794FE14
:102690002A2204210320FEF759FE3A2209210320B1
:1026A000FEF71AFE00F0B8FD212201210420FEF7FA
:1026B0004DFE17A203210420FEF77EFE22220421F4
:1026C0000846FEF743FE3A2209210420FEF704FEE5
:1026D0001248007850B9232206210420FEF736FE66
:1026E000242207210420FEF731FE09E025220621DD
:1026F0000420FEF72BFE262207210420FEF726FEEB
:1027000010BD000043000020202000003A200000FF
:1027100020202020000000002000000042000020B7
:1027200010B500BF0A210120FEF7A4FBC0F58050C0
:1027300084B204EB441101EB4100C11700EB1151CD
:1027400009130D4A11801046B0F90000632801DB1F
:10275000632002E00848B0F90000074908800846F5
:10276000B0F9002005A10748FDF73EFD054A0B2101
:102770000120FEF721FE10BD200000202564252544
:10278000202000008800002010B5FE4800780128B5
:102790001BD0FC480078022817D0FA48007803289C
:1027A00013D0F848007804280FD0F64800780528A0
:1027B0000BD0F4480078062807D0F24800780728A4
:1027C00003D0F0480078082854D1002203210120CA
:1027D000FEF7BCFD012205211046FEF7B7FD0222DF
:1027E00007210120FEF7B2FDE7A201210220FEF73A
:1027F000E3FD032211460220FEF7A8FD0422052175
:102800000220FEF7A3FD052207210220FEF79EFD10
:10281000112201210320FEF799FD1222022103203B
:10282000FEF794FD1F2203210846FEF78FFD2022AC
:1028300004210320FEF78AFD3A2209210320FEF736
:102840004BFD152201210420FEF780FD16220221F6
:102850000420FEF77BFD1F2203210420FEF776FDF6
:10286000202204210846FEF771FD3A2209210420A6
:10287000FEF732FDC3480078092807D0C148007828
:102880000A2803D0BF4800780B284AD11D22012115
:102890000846FEF75BFD1E2202210120FEF756FDD1
:1028A0001F2203210120FEF751FD202204210120D7
:1028B000FEF74CFDB5A209210120FEF77DFD29227E
:1028C00001210220FEF742FD2A2202210846FEF7DE
:1028D0003DFD2B2203210220FEF738FD2C2204218E
:1028E0000220FEF733FD3A2209210220FEF7F4FC14
:1028F000172201210320FEF729FD182202210320BF
:10290000FEF724FD2B2203210846FEF71FFD2C2293
:1029100004210320FEF71AFD3A2209210320FEF7C5
:10292000DBFC98480078012860D19948007828B1EC
:1029300095A203210120FEF73FFD57E0954802785C
:1029400095A19648FDF750FC944A01210846FEF7F0
:1029500033FD9048427892A19048FDF745FC8F4A9C
:1029600007210120FEF728FD8A4882788CA18B4838
:10297000FDF73AFC894A0B210120FEF71DFD854831
:10298000C27887A18548FDF72FFC844A03210220E5
:10299000FEF712FD7F48027981A18048FDF724FCF3
:1029A0007E4A07210220FEF707FD7A4842797CA182
:1029B0007A48FDF719FC794A0B210220FEF7FCFC4E
:1029C0007848027878A17548FDF70EFC734A0B2110
:1029D0000320FEF7F1FC764876A102686F48FDF708
:1029E00003FC6E4A0B210420FEF7E6FC65480078E4
:1029F000022860D16648007828B163A2072101202F
:102A0000FEF7DAFC57E06348027863A16348FDF7FC
:102A1000EBFB624A01210846FEF7CEFC5D48427896
:102A20005FA15E48FDF7E0FB5C4A07210120FEF74D
:102A3000C3FC584882785AA15848FDF7D5FB574A3D
:102A40000B210120FEF7B8FC5248C27854A153482C
:102A5000FDF7CAFB514A03210220FEF7ADFC4D48A9
:102A600002794FA14D48FDF7BFFB4C4A07210220D8
:102A7000FEF7A2FC4748427949A14848FDF7B4FB5C
:102A8000464A0B210220FEF797FC4648027846A1F1
:102A90004248FDF7A9FB414A0B210320FEF78CFCBD
:102AA000434844A102683D48FDF79EFB3B4A0B2189
:102AB0000420FEF781FC33480078032860D13448B5
:102AC000007828B130A20B210120FEF775FC57E0F9
:102AD0003048027830A13148FDF786FB2F4A0121AA
:102AE0000846FEF769FC2B4842782DA12B48FDF7DC
:102AF0007BFB2A4A07210120FEF75EFC25488278ED
:102B000027A12648FDF770FB244A0B210120FEF780
:102B100053FC2048C27822A12048FDF765FB1F4ADC
:102B200003210220FEF748FC1A4802791CA11B4829
:102B3000FDF75AFB194A07210220FEF73DFC154814
:102B4000427917A11548FDF74FFB144A0B210220CB
:102B5000FEF732FC1348027813A11048FDF744FB3E
:102B60000E4A0B210320FEF727FC114811A1026831
:102B70000A48FDF739FB094A0B210420FEF71CFC2B
:102B800000481BE054000020202000003A200000F4
:102B9000440000203A000020253464008800002012
:102BA000253264002C000020256443202000000012
:102BB000300000202564252520200000007804280E
:102BC00069D1FE48007830B1AFF2440203210220FF
:102BD000FEF7F2FB5FE0FA480278AFF24401F948F1
:102BE000FDF702FBF74A01210846FEF7E5FBF44832
:102BF0004278AFF25401F348FDF7F6FAF14A0721A3
:102C00000120FEF7D9FBEE488278AFF26C01ED4867
:102C1000FDF7EAFAEB4A0B210120FEF7CDFBE8486D
:102C2000C278AFF28401E748FDF7DEFAE54A0321F6
:102C30000220FEF7C1FBE2480279AFF29C01E148B5
:102C4000FDF7D2FADF4A07210220FEF7B5FBDC4888
:102C50004279AFF2B401DB48FDF7C6FAD94A0B213D
:102C60000220FEF7A9FBD8480278AFF2C401D5488C
:102C7000FDF7BAFAD34A0B210320FEF79DFBD34898
:102C8000AFF2D0010268CF48FDF7AEFACD4A0B2172
:102C90000420FEF791FBCE480078052869D1C7488B
:102CA000007830B1AFF2201207210220FEF784FB3A
:102CB0005FE0C3480278AFF22011C248FDF794FAF2
:102CC000C04A01210846FEF777FBBD484278AFF2C3
:102CD0003011BC48FDF788FABA4A07210120FEF7F7
:102CE0006BFBB7488278AFF24811B648FDF77CFA23
:102CF000B44A0B210120FEF75FFBB148C278AFF266
:102D00006011B048FDF770FAAE4A03210220FEF7C9
:102D100053FBAB480279AFF27811AA48FDF764FA89
:102D2000A84A07210220FEF747FBA5484279AFF2E7
:102D30009011A448FDF758FAA24A0B210220FEF791
:102D40003BFBA1480278AFF2A0119E48FDF74CFA78
:102D50009C4A0B210320FEF72FFB9C48AFF2AC11DD
:102D600002689848FDF740FA964A0B210420FEF7C6
:102D700023FB97480078062869D19048007830B145
:102D8000AFF2FC120B210220FEF716FB5FE08C482D
:102D90000278AFF2FC118B48FDF726FA894A01212F
:102DA0000846FEF709FB86484278AFF20C218548B9
:102DB000FDF71AFA834A07210120FEF7FDFA804841
:102DC0008278AFF224217F48FDF70EFA7D4A0B216D
:102DD0000120FEF7F1FA7A48C278AFF23C21794837
:102DE000FDF702FA774A03210220FEF7E5FA74485C
:102DF0000279AFF254217348FDF7F6F9714A0721C1
:102E00000220FEF7D9FA6E484279AFF26C216D4884
:102E1000FDF7EAF96B4A0B210220FEF7CDFA6A486A
:102E20000278AFF27C216748FDF7DEF9654A0B2195
:102E30000320FEF7C1FA6548AFF2882102686148B5
:102E4000FDF7D2F95F4A0B210420FEF7B5FA60487E
:102E50000078072869D15948007830B1AFF2D822FC
:102E60000B210320FEF7A8FA5FE055480278AFF285
:102E7000D8215448FDF7B8F9524A01210846FEF717
:102E80009BFA4F484278AFF2E8214E48FDF7ACF983
:102E90004C4A07210120FEF78FFA49488278AFF2A9
:102EA00000314848FDF7A0F9464A0B210120FEF702
:102EB00083FA4348C278AFF218314248FDF794F9DB
:102EC000404A03210220FEF777FA3D480279AFF22B
:102ED00030313C48FDF788F93A4A07210220FEF7D5
:102EE0006BFA37484279AFF248313648FDF77CF942
:102EF000344A0B210220FEF75FFA33480278AFF222
:102F000058313048FDF770F92E4A0B210320FEF7A7
:102F100053FA2E48AFF2643102682A48FDF764F98B
:102F2000284A0B210420FEF747FA29480078082890
:102F300076D12248007830B1AFF2B4320B210420B0
:102F4000FEF73AFA6CE01E480278AFF2B4311D4841
:102F5000FDF74AF91B4A01210846FEF72DFA1848E9
:102F60004278AFF2C4311748FDF73EF9154A072100
:102F70000120FEF721FA12488278AFF2DC311148C5
:102F8000FDF732F90F4A0B210120FEF715FA0C4824
:102F9000C278AFF2F4310B48FDF726F9094A032154
:102FA0000220FEF709FA06480279AFF20C41054803
:102FB000FDF71AF9034A072102200BE04400002024
:102FC0003A000020880000202C0000203000002063
:102FD00054000020FEF7F0F957484279AFF2404123
:102FE0005648FDF701F9554A0B210220FEF7E4F996
:102FF00053480278AFF250415048FDF7F5F84F4A78
:103000000B210320FEF7D8F94E48AFF25841026871
:103010004A48FDF7E9F8494A0B210420FEF7CCF9AC
:1030200049480078092829D14848007828B148A2A1
:103030000B210120FEF7C0F920E04648028846A196
:103040003E48FDF7D1F83D4A0B210120FEF7B4F9C7
:103050004348028843A13948FDF7C6F8374A0B2197
:103060000220FEF7A9F94148028841A13348FDF743
:10307000BBF8324A0B210320FEF79EF93248007854
:103080000A2829D13148007828B131A20B21022029
:10309000FEF792F920E02F4802882FA12748FDF77C
:1030A000A3F8264A0B210120FEF786F92C48028856
:1030B0002CA12248FDF798F8204A0B210220FEF7A8
:1030C0007BF92A4802882AA11C48FDF78DF81B4A83
:1030D0000B210320FEF770F91B4800780B282AD13A
:1030E0001A48007830B1AFF260520B210320FEF78E
:1030F00063F920E01748028817A11048FDF774F81B
:103100000E4A0B210120FEF757F91548028815A138
:103110000A48FDF769F8094A0B210220FEF74CF92D
:103120001248028812A10548FDF75EF8034A0B21F8
:103130000320FEF741F910BD3A000020880000206E
:103140002C0000203000002054000020440000200B
:103150002020200034000020253264636D00000030
:10316000360000202533646D696E000038000020B1
:10317000253264252500000010B50D490D48FDF7E6
:103180001CFD0C4802780CA10D48FDF72DF80C4AE7
:103190000B210320FEF710F90548027809A1084821
:1031A000FDF722F8064A0B210420FEF705F910BDB1
:1031B0002B0000202A00002025644320200000006E
:1031C00088000020256425252020000010B5FDF78B
:1031D0006BFE044601F006F800B20B490880084671
:1031E000B0F90000632801DD632008800648B0F9CB
:1031F000002006A10748FCF7F7FF064A0B21022032
:10320000FEF7DAF810BD00002200002025326463CA
:103210006D0000008800002010B50648B0F90020BD
:1032200005A10748FCF7E0FF054A0B210320FEF744
:10323000C3F810BD2600002025646D696E200000D3
:103240008800002008B501210420FEF729F901219A
:103250000420FEF725F901210420FEF721F9802042
:10326000ADF8000010208DF8030003208DF8020057
:1032700069460F48FDF7E5FC4020ADF8000010203E
:103280008DF8030003208DF8020069460848FDF719
:10329000D8FC2020ADF8000010208DF8030003209A
:1032A0008DF8020069460248FDF7CBFC08BD00001E
:1032B0000008014010B5FFF7C5FF10BD10B58D2007
:1032C00000F048F812490870892000F043F81049CE
:1032D0004870872000F03EF80D498870852000F086
:1032E00039F80B49C870832000F034F80849087198
:1032F000812000F02FF8064948718B2000F02AF851
:103300000349887107210248FFF76DF810BD0000DE
:103310001600002070B5002400F03AF8002512E0F5
:10332000641040210A48FDF75FFD012801D144F0F7
:10333000800480210648FDF762FD80210448FDF7E6
:103340005CFD681CC5B2082DEADB204670BD00009C
:103350000008014070B50446002520210B48FDF708
:103360004CFD80210948FDF748FD20210748FDF765
:1033700046FD204600F06CF8FFF7CCFF0546202103
:103380000248FDF73AFD284670BD000000080140E4
:1033900008B501210420FEF783F84020ADF80000B5
:1033A00048208DF8030069460148FDF74AFC08BD36
:1033B0000008014008B501210420FEF771F8402003
:1033C000ADF8000010208DF8030003208DF80200F6
:1033D00069460248FDF735FC08BD000000080140C1
:1033E00010B507211948FFF711F800218E2000F0D1
:1033F00051F8164801788C2000F04CF813484178B9
:10340000882000F047F811488178862000F042F8C3
:103410000E48C178842000F03DF80C4801798220E4
:1034200000F038F809484179802000F033F8074867
:1034300081798A2000F02EF880218E2000F02AF871
:1034400007210248FEF7CFFF10BD00003A00002020
:1034500070B50446FFF7AEFF002516E004F001004A
:1034600020B140210A48FDF7CAFC03E0402108488A
:10347000FDF7C3FC641080210548FDF7C0FC8021E6
:103480000348FDF7BAFC681CC5B2082DE6DB70BD29
:103490000008014070B505460C4620210A48FDF79A
:1034A000ACFC80210848FDF7A8FC20210648FDF768
:1034B000A6FC2846FFF7CCFF2046FFF7C9FF2021D6
:1034C0000148FDF79AFC70BD0008014008B54FF4B3
:1034D000A060FDF705FE1E208DF8000000208DF88D
:1034E00001008DF8020001208DF803006846FDF709
:1034F000BFFD08BD10B5FE480068D0B90A20FEF730
:10350000B7FFFB480068A0B900BFF9480068002871
:10351000FBD0F848007860B9F748007880F00100E7
:10352000F549087008460078012802D10020F349C7
:103530000860EF48001D006800283AD10A20FEF715
:1035400097FFEB48001D0068002832D100BFE84813
:10355000001D00680028FAD0E748007838B900203C
:10356000E6490860E3480078401CE2490870E148F9
:10357000007801280CD1FFF7A1FE002004E0E0490B
:10358000095CE04A1154401C0628F8DBFDF7B2FD47
:10359000D8480078092803D1FFF722FFFDF7AAFDDC
:1035A000D44800780C2804DBFDF7A4FD0020D149A5
:1035B0000870CF480830006800287DD10A20FEF747
:1035C00057FFCB48083000680028F6D119E00220E8
:1035D000FEF74EFFCC48B0F9000040F67F4188422C
:1035E00009DAC5480078012805D1C7480088401C81
:1035F00000B2C5490880C448008881B2C348FEF7BC
:103600002CFBBB48083000680028E0D0B94800789F
:10361000012804D1BB480078401CBA490870B5485D
:103620000078022808D1B74840780C2804DAB54859
:103630004078401CB3494870AE48007803286DD1EB
:10364000B04880781F2821DAAE484078012817D08A
:10365000AC484078032813D0AA48407805280FD0FA
:10366000A848407807280BD0A6484078082807D0FB
:10367000A44840780A2803D0A24840780C2805D1F5
:10368000A0488078401C9F49887047E09D4880781A
:103690001E2817DA9B48407804280BD099484078B8
:1036A000062807D097484078092803D095484078E5
:1036B0000B2807D1934800E094E08078401C9149A2
:1036C00088702BE08F4989781D291EDA8D4908788A
:1036D000C11700EB91718910A0EB810139B98949BB
:1036E0000978642291FBF2F302FB131139B9854981
:1036F0000978642291FBF2F302FB131129B9814886
:103700008078401C7F49887008E07E4880781C28BB
:1037100004DA7C488078401C7A49887075480078C3
:10372000042808D17748C078182804DA7548C0788A
:10373000401C7449C8706F480078052808D171484A
:1037400000793C2804DA6F480079401C6D49087103
:1037500068480078062808D16A4840793C2804DA8D
:1037600068484079401C67494871624800780728DA
:1037700008D167480078632804DA65480078401C5F
:10378000634908705B480078082808D161480068E0
:10379000632804D25F480068401C5E4908605548B1
:1037A0000078092808D15C480088632804DA5A4860
:1037B0000088401C584908804E4800780A2804D1E7
:1037C00056480088401C554908804A4800780B2814
:1037D00008D153480088632804DA51480088401C07
:1037E0004F49088042480C30006800287ED10A20EA
:1037F000FEF73EFE3E480C3000680028F6D117E088
:103800000220FEF735FE4048B0F90000002809DD2F
:1038100039480078012805D13B480088401E00B295
:10382000394908803848008881B23848FEF715FACF
:103830002F480C3000680028E2D02E48007801287C
:1038400008D130480078002804DD2E480078401E5A
:103850002C49087027480078022808D12948407868
:10386000002804DD27484078401E2649487021483A
:103870000078032808D123488078002804DD2148F7
:103880008078401E1F4988701A480078042808D1A3
:103890001C48C078002804DD1A48C078401E194929
:1038A000C87014480078052808D116480079002807
:1038B00004DD14480079401E124908710D48007853
:1038C000062808D10F484079002804DD0D484079CA
:1038D000401E0C49487107480078072825D10C483C
:1038E0000078002821DD0A4800781BE050E0000045
:1038F000308121425400002042000020B4012242C5
:10390000160000203A00002028000020002C014072
:103910002C00002030000020340000203600002061
:1039200038000020401E1B4908701B4800780828FA
:1039300007D11A48006820B118480068401E17498E
:10394000086015480078092808D115480088002823
:1039500004DD13480088401E114908800E48007895
:103960000A2808D10F480088002804DD0D48008887
:10397000401E0C490880084800780B2808D10A48E6
:103980000088002804DD08480088401E0649088099
:1039900010BD00002C00002054000020300000204A
:1039A000340000203600002038000020FEF744FDDF
:1039B000FDF757FB4FF4FA70FEF75AFDFDF71CFBBD
:1039C0004FF4165000F006F9FDF71EFC45A2012148
:1039D0000220FDF7F1FCFDF701F8FDF70DFBFDF707
:1039E000B7FAFDF777F8FFF765FC47214FF4486019
:1039F000FDF788FE40F2CF216320FDF755FFFDF76C
:103A000079FB6EE0FFF776FD3B48007800285ED139
:103A1000FEF79CFDFEF7B8FE3848006800284BD141
:103A200037480078C8BB374800883749B1F90010DB
:103A3000401A40F67F414843632190FBF1F000B209
:103A4000324908800846B0F90000002801DA002059
:103A500008802E48008881B22D48FEF7FEF82D48D8
:103A600000782D490968884213D82C4800782C49E1
:103A7000097888420DDC2B48B0F900002A490988F2
:103A8000884206DB2948B0F90000294909888842A4
:103A900004DD01202749086019E003E000202549E2
:103AA000086014E01948008881B21948FEF7D5F87B
:103AB0000020204908600AE010480068012806D16B
:103AC00000201C49086000211148FEF7C6F80A488A
:103AD000007808B1FEF758FEFEF76AFA1420FEF7E8
:103AE000C7FC8FE72020204C6F6164696E672E2E23
:103AF0002E202020000000005400002000812142E0
:103B00004200002038000020200000202800002073
:103B1000002C01402B000020300000202A00002053
:103B20002C0000202200002034000020260000206D
:103B300036000020B401224210B5FFF7BFFB214838
:103B4000027821A12148FCF74FFB204A01210846B9
:103B5000FDF732FC1B4842781DA11C48FCF744FBD2
:103B60001A4A07210120FDF727FC1648827818A180
:103B70001648FCF739FB154A0B210120FDF71CFC08
:103B80001048C27812A11148FCF72EFB0F4A0321FE
:103B90000220FDF711FC0B4802790DA10B48FCF740
:103BA00023FB0A4A07210220FDF706FC054842795B
:103BB00007A10648FCF718FB044A0B210220FDF779
:103BC000FBFB10BD16000020253464008800002097
:103BD0002532640010B586B00446012144F2050088
:103BE000FDF75EFC2848FEF7D1F84FF40070ADF801
:103BF000140003208DF8160018208DF8170005A971
:103C00002248FDF71EF84FF48060ADF81400042040
:103C10008DF8170005A91D48FDF713F825208DF82C
:103C2000000003208DF8010002208DF80200012021
:103C30008DF803006846FDF71BFA01940020ADF8EB
:103C40000800ADF80A00ADF80C00ADF810000C202B
:103C5000ADF80E0001A90C48FEF736F901A90A4893
:103C6000FEF732F9012240F225510748FEF706F926
:103C7000002240F224410448FEF700F901210248E5
:103C8000FEF777F806B010BD00380140000801408B
:103C9000FF2912D00BE000BF104A128802F0400248
:103CA000002AF9D002780D4B1B1D1A80401C0A0017
:103CB000A1F10103D9B2EED10FE00BE000BF074A3A
:103CC000128802F04002002AF9D00278034B1B1D33
:103CD0001A80401C0278002AF0D170470038014059
:103CE00010B500290AD00878002807D00548784484
:103CF000FCF73EFD002801D0002010BD02487844AA
:103D000010BD0000261800001E18000021F000421F
:103D1000A2F16052B2F5801F01F0004328BFD2F13A
:103D20007F6C0BD95FEA001C43EAC20242EB507081
:103D300018BF704728BF20F001007047B2F5801F00
:103D4000BCBF184670474FEA410C1CF5001F02D259
:103D5000084600F0BCBA70B500F062F900000089B6
:103D6000FFF7F6BF4FF00040A0F58000704700005D
:103D70002DE9C04130B4DFF8A0C23CEA111418BFED
:103D80003CEA131400F0EC8081EA03051CEA1114EC
:103D900044EAD57418BF1CEA131500F0C780A4EBE1
:103DA00005044FF0004545EAC12145EAC32341EA35
:103DB000505143EA525304F17F74994204F50034A0
:103DC0004FEAC0204FEAC22208BF904200F09C8018
:103DD0004FEA13650FF24016765D4FEA134506FB76
:103DE00005F7C7F1807706FB07F74FEAD737A7FB40
:103DF00003687642C8F58038A7FB06CE38BFA8F125
:103E0000010807FB08E64FF0000EA6FB028CE6FB5C
:103E100003CEDCF1000CCEF1004E38BFAEF1010E46
:103E2000A6FB0C584FF000074FF00005E6FB0E878D
:103E3000A1FB08C6A0FB07CE16EB0E0645F1000558
:103E4000E1FB076515F1E04E7EBFA4F580345FEA23
:103E500046066D4116F1800745F100054FEA172728
:103E60004FEA066647EA0567A6F1DE46B6F1805FCF
:103E70004FEA15251FD9384624F0010C05EBC47113
:103E8000BCF1FE6F01EB0C1102D8F0BCBDE8008163
:103E900024425CBF01F5801E9EEAC47F02D4F0BCC0
:103EA000BDE80081244238D4F0BCA1F1C041BDE896
:103EB000004100F003B94FEAD22242EA43524FEAEE
:103EC000D323A7FB02864FEAD02040EA415007FBEC
:103ED00003661EEA0E0F4FEAD12105FB026658BFAA
:103EE000A6EB0056B6EB00564FEA520E4EEAC37EE2
:103EF00018EB0E0E56EB530EBDD518EB02085E41C3
:103F00007F1C55F10005B6E74FF480154FF0000710
:103F10004FF000064FF00008ADE7F0BC4FF0000096
:103F200001F1C04101F00041BDE8008111EA0C1F20
:103F30000CEA131500D00CE013EA0C1F00F02580EA
:103F40004FF00000F0BC81EA030101F00041BDE840
:103F50000081F0BCBDE8004181EA030100F0AEB889
:103F6000F0BCBDE8004170B500F05AF8097EFC3E97
:103F700000F007B881EA03014FF0000001F00041B2
:103F8000704781EA030100F099B8F0BCBDE8004138
:103F90004FF0000021497047FFFDFBF9F7F5F4F2FF
:103FA000F0EEEDEBE9E8E6E4E3E1E0DEDDDBDAD8D4
:103FB000D7D5D4D3D1D0CFCDCCCBCAC8C7C6C5C432
:103FC000C2C1C0BFBEBDBCBBBAB9B8B7B6B5B4B349
:103FD000B2B1B0AFAEADACABAAA9A8A8A7A6A5A434
:103FE000A3A3A2A1A09F9F9E9D9C9C9B9A999998F8
:103FF0009797969595949393929191908F8F8E8E9B
:104000008D8C8C8B8B8A8989888887878685858427
:1040100084838382828181800000FF070000F87F13
:104020000EF1020E2EF0030E5EF8046B364205D43C
:10403000012A43EB030515F5001F12D8012841EBB7
:10404000010C1CF5001F0CD80ED14FEAD17C15F5E0
:10405000001F0CEB4C0C0CF1020C08BF4CEBD37C9A
:1040600004E04FF0080C01E04FEAD37C0CEB4C0568
:1040700026FA05F606F00706B6F1040C06D20EEB9A
:10408000860CBDE870404CF0010C6047DFE80CF096
:10409000090B02024FF000414FF00000A1F5002192
:1040A00070BD19461046012851EB010418BFD4F524
:1040B000001484BF002001F0004170BD0808A0F585
:1040C00000114FEA3101704743004FEAD30C4FEA29
:1040D0003C0C43401FBF40070CF1605113F0FE4FF2
:1040E00070471CF0006F03D100200CF000417047B6
:1040F0000CF0004343EA507010B540EACC0000F0E9
:10410000A0F800BF000000924FEA0001FFF7D6BF01
:104110004FF000414FF00000A1F500217047000072
:1041200090EA010F48BF81F0004100F1DC80421AA3
:104130003CBF801A89184FEAD0524FF07F4C1CEADE
:10414000410FA2EBD15318BF9CEA026F00F03B80F5
:104150004FF0004C4CEA00204CEA012121FA03FC0C
:1041600010EB0C0C1ED202F1FF325FEA1C2040EB78
:10417000C25038BF70471CF07F0F4FEA400C18BF89
:10418000BCF17F4F38BF7047C3F12003994008BF8F
:1041900020F00100BCF17F4F38BF7047A0F1C04054
:1041A00000F095B84FEA3C00000A40EBC25028BF2F
:1041B0001CF0FF0F4FEA400CE6D018BFBCF17F4F58
:1041C00038BF7047EAE79CEA026F05D010EA5C0F3F
:1041D00008BF00F00040704710B500F032F800BF93
:1041E00064FBBE3E41000B0ED3F19E0208D950F491
:1041F00000034FEA032323FA02F048BF404270470E
:1042000010B500F01EF800BF4992248000207047CE
:104210006FF0004282EA200070470000B0FA80F39D
:1042200010FA03F2C3F19D030AD0D90501EB122065
:10423000530638BF704700F1010008BF20F00100AD
:1042400070470EF1020E2EF0030E5EF8044B24426E
:1042500004D44FEA4102B2F17F4F11D84FEA400334
:10426000B3F17F4F0CD80ED14FEAD07CB2F17F4F23
:104270000CEB4C0C0CF1020C08BF4CEBD17C04E0B5
:104280004FF0080C01E04FEAD17C0CEB4C0324FA10
:1042900003F404F00704B4F1040C06D20EEB840C12
:1042A000BDE810404CF0010C6047DFE80CF0070857
:1042B00002024FF00040A0F5800010BD0846420009
:1042C00018BFD2F1807288BF00F0004010BDFF21FE
:1042D00041EAD050C005704790EA010F48BF81F015
:1042E00000413FF524AF421A04D882F00042A0EB0F
:1042F000020011444FEAD0524FF07F4C1CEA410FAC
:10430000A2EBD15318BF9CEA026F4AD04FF0004C89
:104310004CEA00204CEA012121FA03FCB0EB0C0C22
:104320000FD412F0FE0F36D05FEA4C001DD50012FC
:1043300040EBC25038BF70471CF03F0F18BF7047AA
:104340000BE0A2F101025FEA1C2040EBC25038BF33
:1043500070471CF07F0F18BF7047C3F120039940CE
:1043600014BF401E20F00100704780084FEA12235E
:1043700008BF7047B0FA80FCA2EB0C02CCF1280C0D
:1043800060FA0CF093EA122F04BF00EBC2507047A2
:104390004FEAC3707047130A5FEADC1008BF70472A
:1043A000F6E79CEA026F04D010EA5C0F08BF002019
:1043B000704710B5FFF745FF40DFF63E81F0004043
:1043C0007047000000000000000000000000000036
:1043D0000000000000F80000000000000033300082
:1043E000000000100C06100C060000000000000089
:1043F000000040C07840C0784000043F04043F04FF
:104400000400007088FC08300000001820FF211E06
:104410000000F008F000E018000000211C031E213D
:104420001E0000F00888700000001E2123241927B8
:10443000211010160E000000000000000000000017
:104440000000000000E0180402000000000718202F
:10445000400000020418E00000000040201807009F
:104460000000404080F0804040000202010F010245
:104470000200000000F0000000000101011F010126
:104480000100000000000000000080B0700000008B
:104490000000000000000000000000010101010117
:1044A00001010000000000000000003030000000AA
:1044B0000000000000008060180400601806010081
:1044C000000000E010080810E000000F102020108D
:1044D0000F00001010F8000000000020203F2020F6
:1044E000000000700808088870000030282422218D
:1044F0003000003008888848300000182020201143
:104500000E000000C02010F8000000070424243F23
:10451000240000F8088888080800001921202011CC
:104520000E0000E0108888180000000F11202011F4
:104530000E0000380808C83808000000003F0000DE
:1045400000000070880808887000001C22212122C9
:104550001C0000E010080810E000000031222211C9
:104560000F00000000C0C00000000000003030005C
:1045700000000000008000000000000080600000DB
:104580000000000080402010080000010204081014
:104590002000404040404040400004040404040423
:1045A00004000008102040800000002010080402D1
:1045B0000100007048080808F000000000303601D3
:1045C0000000C030C828E810E00007182724231492
:1045D0000B000000C038E0000000203C230202274E
:1045E000382008F8888888700000203F202020119B
:1045F0000E00C030080808083800071820202010D6
:10460000080008F808080810E000203F20202010CB
:104610000F0008F88888E8081000203F2020232099
:10462000180008F88888E8081000203F20000300E0
:104630000000C03008080838000007182020221E9B
:10464000020008F808000008F808203F21010121B5
:104650003F20000808F8080800000020203F202024
:10466000000000000808F8080800C08080807F0073
:10467000000008F888C028180800203F20012638CC
:10468000200008F8080000000000203F2020202023
:10469000300008F8F800F8F80800203F003F003F1D
:1046A000200008F830C00008F808203F2000071854
:1046B0003F00E01008080810E0000F102020201034
:1046C0000F0008F808080808F000203F2101010148
:1046D0000000E01008080810E0000F1824243850EB
:1046E0004F0008F8888888887000203F2000030C5D
:1046F0003020007088080808380000382021212266
:104700001C00180808F8080818000000203F2000C6
:10471000000008F808000008F808001F20202020EA
:104720001F000878880000C83808000007380E010C
:104730000000F80800F80008F800033C0700073CF8
:104740000300081868808068180820302C03032CA8
:1047500030200838C800C83808000000203F20007A
:10476000000010080808C83808002038262120203A
:104770001800000000FE020202000000007F40401E
:104780004000000C30C000000000000000010638AE
:10479000C00000020202FE000000004040407F0016
:1047A00000000000040202020400000000000000FB
:1047B00000000000000000000000808080808080F9
:1047C00080800002020400000000000000000000E1
:1047D0000000000080808080000000192422222236
:1047E0003F2008F8008080000000003F11202011C9
:1047F0000E000000008080800000000E11202020AC
:104800001100000000808088F800000E11202010A8
:104810003F200000808080800000001F2222222292
:104820001300008080F0888888180020203F202016
:1048300000000000808080808000006B949494933E
:10484000600008F8008080800000203F21000020E8
:104850003F2000809898000000000020203F20208A
:104860000000000000809898000000C08080807FD9
:10487000000008F8000080808000203F24022D30D6
:104880002000000808F8000000000020203F202041
:1048900000008080808080808000203F20003F20BA
:1048A000003F8080008080800000203F21000020A9
:1048B0003F200000808080800000001F20202020FA
:1048C0001F00808000808000000080FFA120201158
:1048D0000E000000008080808000000E112020A0CB
:1048E000FF80808080008080800020203F21200089
:1048F0000100000080808080800000332424242474
:104900001900008080E0808000000000001F20204F
:1049100000008080000000808000001F2020201008
:104920003F20808080000080808000010E300806DB
:10493000010080800080008080800F300C030C30EC
:104940000F0000808000808080000020312E0E311A
:104950002000808080000080808080818E7018061A
:10496000010000808080808080000021302C222186
:10497000300000000000807C020200000000003FC8
:10498000404000000000FF00000000000000FF00A9
:1049900000000002027C800000000040403F000058
:1049A00000000006010102020404000000000000F3
:1049B0000000002018C744444444FC4444444404D8
:1049C00000000000000000000000000000000000E7
:1049D00000000404040704040404FF0404040404A1
:1049E00004000000000000000000000000000000C3
:1049F0000000000000FE2222222222222222FE00AB
:104A000000000000000000000000000000000000A6
:104A100000008040300F02020202020242827F0048
:104A20000000000000000000000000000000000086
:104A30000000000000FE82828282828282FE0000EC
:104A40000000000000000000000000000000000066
:104A50000000000000FF40404040404040FF000098
:104A60000000000000000000000000000000000046
:104A7000000000FC848484FC001010101010FF1053
:104A80001000000000000000000000000000000016
:104A90000000003F1010103F0000010640807F0022
:104AA0000000000000000000000000000000000006
:104AB0000000804020908886808080838C10204079
:104AC0008000000000000000000000000000000066
:104AD0000000008040201807004080403F00000098
:104AE00000000000000000000000000000000000C6
:104AF00000002424A4FE232200C03800FF00081078
:104B00006000000000000000000000000000000045
:104B10000000080601FF01068180404027100C03B9
:104B20000000000000000000000000000000000085
:104B30000000000000BE2A2A2AEA2A2A2A3E000093
:104B40000000000000000000000000000000000065
:104B50000000004442494949497F49494949414087
:104B60000000000000000000000000000000000045
:104B700000000004FF242424FF0400FE222222FE61
:104B80000000000000000000000000000000000025
:104B9000000088482F090919AF48300F0242827F70
:104BA0000000000000000000000000000000000005
:104BB00000008080808080808080808080808080F5
:104BC0008000000000000000000000000000000065
:104BD00000000000000000000000000000000000D5
:104BE00000000000000000000000000000000000C5
:104BF000000000000808080808080808080808005D
:104C000000000000000000000000000000000000A4
:104C100000001010101010101010101010101010B4
:104C20001000000000000000000000000000000074
:104C300000000004848484848484848484848404C0
:104C40000000000000000000000000000000000064
:104C50000000202020202020202020202020202094
:104C60002000000000000000000000000000000024
:104C7000000000FC040404FC040404FC040404FC20
:104C80000000000000000000000000000000000024
:104C90000000007F28242320202020212222227FA0
:104CA0000000000000000000000000000000000004
:104CB00000000002424242C27E42424242C202021E
:104CC00000000000000000000000000000000000E4
:104CD000000040404040784740404040407F4040D6
:104CE0004000000000000000000000000000000084
:104CF000000020202020202021222C2020202020E5
:104D00002000000000000000000000000000000083
:104D10000000004020100C03000000010204186095
:104D20000000000000000000000000000000000083
:104D30000000000000FE82828282828282FE0000E9
:104D40000000000000000000000000000000000063
:104D50000000000000FF40404040404040FF000095
:104D60000000000000000000000000000000000043
:104D70000000048484FC848400040484E41C84040F
:104D8000040000000000000000000000000000001F
:104D900000002060201F101004020100FF0000012D
:104DA00006000000000000000000000000000000FD
:104DB00000001010FF101020A4ACB5A6B4ACA420C5
:104DC00020000000000000000000000000000000C3
:104DD000000010301F0888804F3A0A0A7A8A8F80B4
:104DE000E0000000000000000000000000000000E3
:104DF00000001060028C0000FE9292929292FE00DF
:104E000000000000000000000000000000000000A2
:104E1000000004047E01407E42427E427E42427E89
:104E20004000000000000000000000000000000042
:104E300000000000FC242424FC252624FC24242437
:104E4000040000000000000000000000000000005E
:104E5000000040308F80844C55252525554C80809E
:104E600080000000000000000000000000000000C2
:104E70000000048484FC848400040484E41C84040E
:104E8000040000000000000000000000000000001E
:104E900000002060201F101004020100FF0000012C
:104EA00006000000000000000000000000000000FC
:104EB00000001010FF101020A4ACB5A6B4ACA420C4
:104EC00020000000000000000000000000000000C2
:104ED000000010301F0888804F3A0A0A7A8A8F80B3
:104EE000E0000000000000000000000000000000E2
:104EF00000001060028C00FE929292929292FE004C
:104F000000000000000000000000000000000000A1
:104F1000000004047E014448507F40407F504844D4
:104F20004000000000000000000000000000000041
:104F300000000000FC242424FC252624FC24242436
:104F4000040000000000000000000000000000005D
:104F5000000040308F80844C55252525554C80809D
:104F600080000000000000000000000000000000C1
:104F700000004040424458C0407F40C05048464036
:104F800040000000000000000000000000000000E1
:104F900000008080402018070000003F4040404053
:104FA0007800000000000000000000000000000089
:104FB000000000FE424242FE0042A29E82A2C2BE09
:104FC00000000000000000000000000000000000E1
:104FD0000000806F080828CF00002FC8080828CFDD
:104FE00000000000000000000000000000000000C1
:104FF000000002E222223E00809E9292F292929E55
:105000008000000000000000000000000000000020
:105010000000004382423E40474444447F4444549D
:10502000E700000000000000000000000000000099
:1050300000000000FC242424FC252624FC24242435
:10504000040000000000000000000000000000005C
:10505000000040308F80844C55252525554C80809C
:1050600080000000000000000000000000000000C0
:1050700000000080601E20C000FF0080601E20C075
:105080000000000000000000000000000000000020
:105090000000414044444444447F44444444444028
:1050A00040000000000000000000000000000000C0
:1050B00000002021F2080410888447344484940CB2
:1050C00000000000000000000000000000000000E0
:1050D0000000048485945D57242424544C448405A2
:1050E00005000000000000000000000000000000BB
:1050F0000000003E22E2223E00FE2222222222E284
:10510000020000000000000000000000000000009D
:105110000000203F201F1111007F444444444447B5
:10512000400000000000000000000000000000003F
:105130000000040404F484D4A5A6A4D484F40404D4
:10514000040000000000000000000000000000005B
:10515000000000FE0202123A1613121A3242827E38
:10516000000000000000000000000000000000003F
:10517000000000F80122A0A2A222FE22AA3202FE12
:10518000000000000000000000000000000000001F
:10519000000000FF0010130A4B20170C133880FF8B
:1051A00000000000000000000000000000000000FF
:1051B0000000008060F80704E4A4A4BFA4A4E404F1
:1051C00000000000000000000000000000000000DF
:1051D0000000010000FF40407F4A4A4A4A4A7F409F
:1051E000400000000000000000000000000000007F
:1051F00000001010D0FF9014E4AFA4A4A4AFE40406
:10520000000000000000000000000000000000009E
:105210000000040300FF00894B2A1A0E1A2A4B884B
:1052200080000000000000000000000000000000FE
:105230000000101090909090901010FF1010111618
:10524000100000000000000000000000000000004E
:105250000000002060203F10101000030C102040C0
:10526000F800000000000000000000000000000046
:105270000000000000F8888C8A89888888F800007F
:10528000000000000000000000000000000000001E
:105290000000000000FF44444444444444FF000034
:1052A00000000000000000000000000000000000FE
:1052B00000004044C4444444401010FF101010F05B
:1052C00000000000000000000000000000000000DE
:1052D0000000103C131014B840300E014080403FD5
:1052E00000000000000000000000000000000000BE
:1052F000000000002424242424FC22222223220053
:10530000000000000000000000000000000000009D
:105310000000020202020242827F02020202020234
:10532000020000000000000000000000000000007B
:1053300000004044C4444444401010FF101010F0DA
:10534000000000000000000000000000000000005D
:105350000000103C131014B840300E014080403F54
:10536000000000000000000000000000000000003D
:105370000000404042CC000444645C47F444444490
:105380000400000000000000000000000000000019
:1053900000000040201F2044444444447F444444CF
:1053A00044000000000000000000000000000000B9
:1053B00000002030AC6320182024A4243FA424A49F
:1053C000600000000000000000000000000000007D
:1053D0000000226722121212888A4C29180F1828FE
:1053E000C8000000000000000000000000000000F5
:1053F0000000404042CC0040404040FF4040404020
:10540000400000000000000000000000000000005C
:1054100000000000007F2010000000FF00000000DE
:10542000000000000000000000000000000000007C
:10543000000000FC848484FC001010101010FF1089
:10544000100000000000000000000000000000004C
:105450000000003F1010103F0000010640807F0058
:10546000000000000000000000000000000000003C
:105470000000000000000000FF40404040404000AD
:10548000000000000000000000000000000000001C
:1054900000004040404040407F404040404040404D
:1054A00040000000000000000000000000000000BC
:1054B000000000FE225A8600FE9292929292FE0016
:1054C00000000000000000000000000000000000DC
:1054D000000000FF04080700FF4020030C142241D5
:1054E000400000000000000000000000000000007C
:1054F0000000000024560008000000208800000082
:1055000028010008AC560008880000201807000099
:10551000440100081001000043000000F8FFFFFFF5
:1055200000404040404040404040414141414140B6
:10553000404040404040404040404040404040406B
:1055400040050202020202020202020202020202FA
:1055500002202020202020202020200202020202FF
:105560000202909090909090101010101010101057
:105570001010101010101010101010100202020263
:1055800002028888888888880808080808080808A7
:1055900008080808080808080808080802020202A3
:1055A00040000000000000000000000000000000BB
:1055B00000000000000000000000000000000000EB
:1055C00000000000000000000000000000000000DB
:1055D00000000000000000000000000000000000CB
:1055E00000000000000000000000000000000000BB
:1055F00000000000000000000000000000000000AB
:10560000000000000000000000000000000000009A
:10561000000000000000000000000000000000008A
:105620000000000000000000010203040102030466
:105630000607080902040608000019021A0E1600DF
:105640000300000000000000000000000000000057
:105650002D000000230000000A003C004600190253
:105660001A0E1600030000000001000000000000F8
:10567000000000000000000000000000000000002A
:105680000000000000A24A0400000000000000002A
:1056900001020304060708090000000000000000E2
:0C56A000000000000000000000000000FE
:04000005080000ED02
:00000001FF
